:10000000830100308A009928FC0003088301C600A0
:100010000408C7000A08C8008A017008CD007108EA
:10002000CE007208CF007308D0007408D1007508A4
:10003000D2007608D3007708D4007808D500790874
:10004000D6007A08D7007B08D8005A08D9004B0898
:10005000C9004C08CA008B1E47280B1D4728831671
:1000600003173B1839280A168A15E6200A128A1146
:1000700047288312251C42280A168A15C6210A120F
:100080008A1147280A168A15D5210A128A11831661
:1000900003138C1E632883128C1E62288515023080
:1000A00083160317A600321D5D28B2185D280A16B4
:1000B0008A1549220A128A1162280A168A152D23E6
:1000C0000A128A1183160C1E7028831285140230BE
:1000D00083160317A6000A168A15C7200A128A116A
:1000E000031383124D08F0004E08F1004F08F20090
:1000F0005008F3005108F4005208F5005308F600C8
:100100005408F7005508F8005608F9005708FA0097
:100110005808FB005908DA004908CB004A08CC000F
:100120004708840048088A0046088300FC0E7C0EBD
:10013000090083010730CC00C430CB00A03084001C
:10014000DC30A62083010A168A11FB2EF0000A1269
:100150008A11B4200A128A118000840A04087006E9
:10016000031DA7280034CB00CC1BBD284C088A00F7
:100170004B08CB0A0319CC0A820083134C1883174F
:100180004B08CB0A84000008080044344534383456
:100190003634383431342034443465346D346F347B
:1001A0006E347334743472346134743469346F343B
:1001B0006E3420344B346934743400346D34783404
:1001C000733461346C346534733440346D34783452
:1001D00063346F346D342E3463346F346D340034D3
:1001E000733461346C3465347334403463346D3447
:1001F0006C346D346934633472346F342E34633448
:100200006F342E3475346B3400347734773477346C
:100210002E3463346D346C346D3469346334723429
:100220006F342E3463346F342E3475346B340034B1
:10023000733461346C3465347334403463346D34F6
:100240006C346D346934633472346F342E346334F7
:100250006F346D342E3473346734003443344D348A
:100260004C342034533469346E3467346134703420
:100270006F34723465340034423455345334593455
:10028000003443344F344E344E34453443345434C4
:1002900000344534523452344F34523400344E34E6
:1002A0004F34203443344134523452344934453489
:1002B0005234003443344D344C34203455344B34B0
:1002C00000344F344B3400344E3459344934003404
:1002D000523449344E34473400344E344F34203491
:1002E0004434493441344C34203454344F344E3443
:1002F000453400344D3458342D3443344F344D3468
:100300002C34203449344E344334003449346E3470
:10031000763461346C3469346434203443344D347D
:1003200058343834363438342034523465347634E2
:1003300020344334003443344F344E344E34453447
:1003400043345434203431343234303430342F3464
:1003500037343534003443344F344E344E3445341E
:1003600043345434203431343234303430342F3444
:10037000313435343034003443344F344E344E3419
:10038000453443345434203436343034303400343B
:10039000543465346C343A342B34343434342834A3
:1003A0003034293431343634323431342034383432
:1003B00037343534353430343034003443344F340A
:1003C0004E344E344534433454342034323434348F
:1003D00030343034003443344F344E344E344534AA
:1003E00043345434203433343034303400344334E0
:1003F0004F344E344E34453443345434203437343F
:1004000035342F34313432343034303400344334E2
:100410004F344E344E344534433454342034313424
:10042000353430342F3431343234303430340034D5
:1004300043344F344E344E344534433454342034F2
:100440003134323430343034003445344634383486
:100450003634383431342034563432342E34303457
:02046000003466
:10046A00831203132108F0002208F1002308F20086
:10047A002408F30004300A168A1580207008A800A0
:10048A007108A9007208AA007308AB002808F400D2
:10049A002908F5002A08F6002B08F700F0010930B0
:1004AA00F1003D30F2000030F3010A128A11FF26F2
:1004BA000A128A11FF307007A600FF3003180030B5
:1004CA007107A700803AF0008130700200300319EA
:1004DA0026020318722AA71FB22A2108F00022084E
:1004EA00F1002308F2002408F30006300A168A15E0
:1004FA0080207008A8007108A9007208AA00730871
:10050A00AB002808F4002908F5002A08F6002B0891
:10051A00F700F0010930F1003D30F2000030F3013C
:10052A000A128A11FF260A128A11FF307007A600E2
:10053A00FF30031800307107A700803AF0008130BD
:10054A0070020030031926020318AD2AA71FAF2A2A
:10055A000130D22A83161811B42A83161815831269
:10056A0026088316990018128312981718169812DB
:10057A0083160C128C128312A50883160319C72A34
:10058A001817C82A18138312A5080319CE2A181790
:10059A00CF2A1813831698160030831208000F30DA
:1005AA000313831208000F300313831208000F305D
:1005BA000313831208000F300313831208000F304D
:1005CA000313831208000F300313831208008316E3
:1005DA00031792010E3093050030920610309306ED
:1005EA00120883120313AD0083160317130883122C
:1005FA000313AE00E1300A168A1549210A128A113C
:10060A00163083160317A5002508031D092B0A3087
:10061A009206120883120313AD00831603171308F8
:10062A0083120313AE00E1300A168A1549210A1211
:10063A008A11213083160317A5002508031D222BD2
:10064A0000309205FF309305120883120313AD00A0
:10065A0083160317130883120313AE00E1300A1638
:10066A008A1549210A128A11083083160317A30032
:10067A002308031D3D2B0313831208000F300313B5
:10068A00831208000F300313831208000F3003137C
:10069A00831208000F300313831208000F3003136C
:1006AA00831208000F30031383120800E030831608
:1006BA0003179205FF30930583122908F0000310EF
:1006CA00F00C0310F00C0310700C1F3983169206FD
:1006DA00120883120313AD0083160317130883123B
:1006EA000313AE00E1300A168A154921831603174F
:1006FA009416E0309405FF30950583122A08F0001D
:10070A000310F00C0310F00C0310700C1F39831641
:10071A009406140883120313AD00831603171508F1
:10072A0083120313AE00E2300A168A15492983128E
:10073A000313A201A301A4018316031794010E3027
:10074A009505023094061030950614088312031397
:10075A00AD0083160317150883120313AE00E230A7
:10076A000A168A1549210C3083160317A30005308F
:10077A000A168A1108200A128A1183160317321BD5
:10078A00982D28080319982DE6300A168A155E2135
:10079A000A128A11700883160317990071089A00C1
:1007AA00191BD92B0C30A3002308031DBC2B0030C6
:1007BA0094050E309505F8309406D0309506140845
:1007CA0083120313AD00831603171508831203134C
:1007DA00AE00E2300A168A1549210A128A112D3012
:1007EA0083160317A300321B982D28080319982D86
:0607FA002308031DF82B8B
:1008000083122B08F039031D2A2C00308316920521
:100810000E30930518309206C030930612088312EA
:100820000313AD0083160317130883120313AE00DE
:10083000E1300A168A1549210A128A110A308316F4
:100840000317A300321B982D28080319982D23089D
:10085000031D222CFF308316960016088312031303
:10086000AD00E3300A168A15402183160317920162
:100870000E3093057F309206C03093061208831223
:100880000313AD0083160317130883120313AE007E
:10089000E1300A168A1549210A128A1103172B081A
:1008A000F039031D812C1B308316A30005300A1676
:1008B0008A1108200A128A1183160317321B982DF9
:1008C00028080319982DE6300A168A155E210A12A7
:1008D0008A11700883160317990071089A001A1D6F
:1008E000792C9A1C792C83120313A401A40A831671
:1008F00003172308831203130319832CA408031975
:10090000562C83120313A4080319462D05300A162A
:100910008A1108200A128A1183160317321B982D98
:1009200028080319982DE6300A168A155E210A1246
:100930008A11700883160317990071089A009A1893
:10094000862C3C30A300321B982D28080319982DC3
:100950001E3023020318A32C15141408831203134A
:10096000AD0083160317150883120313AE00E2309F
:100970000A168A1549210A128A1183160317321B97
:10098000982D28080319982D0F3023020318BF2C27
:10099000FF3094050F30950500309406F030950631
:1009A000140883120313AD0083160317150883126E
:1009B0000313AE00E2300A168A15492105300A16E3
:1009C0008A1108200A128A1183160317321B982DE8
:1009D00028080319982D83120313A308031D132D50
:1009E000831603172308031D132DFF3092050F30C4
:1009F000930500309206E030930612088312031329
:100A0000AD0083160317130883120313AE00E13001
:100A10000A168A154921143083160317A30083127E
:100A20000313A301A30AE6300A168A155E210A12EF
:100A30008A11700883160317990071089A001A1D0D
:100A4000302D991F302D1A1C302D83120313A2084C
:100A5000031D2E2D86100514A201A20A831603176A
:100A60001A1DDE2C991FDE2C1A1CDE2C8312031398
:100A7000A3080319DE2C83160317321B982D2808B0
:100A80000319982D230803199D2D3D2D03172B08BD
:100A9000F039031D4E2D8316B21D982D1830831684
:100AA000A30005300A168A1108200A128A1183163B
:100AB0000317321B982D28080319982DE6300A16C3
:100AC0008A155E210A128A1170088316031799008D
:100AD00071089A001A1D702D991F702D1A18722D09
:100AE0001830A3002308031D512D8312281D7B2DD0
:100AF000831615147D2D8316151014088312031305
:100B0000AD0083160317150883120313AE00E230FD
:100B10000A168A1549210A128A11861005144D30C9
:100B200083160317A300321B982D2808031D9A2D46
:100B30000330A62D2308031D932D5B230A128A116F
:100B4000A408031DA52D0830A62D0730031383121A
:100B50000800831203179E1FF72D17088316A8009D
:100B6000CE2D9C23C42D0A128A156F200A128A11D9
:100B7000C42D5723C42D5323C42D4F23C42D4B23E1
:100B8000C42D4723C42D4323A100452E0A128A15E4
:100B9000D2200A128A11C42D0430632E83122B082E
:100BA000F039F200F301F32D72080319B12D103A58
:100BB0000319B12D303A0319B32D103A0319B92D89
:100BC000703A0319BB2D103A0319BD2D303A0319A1
:100BD000BF2D103A0319C12DF03A0319C32D103A55
:100BE0000319C62DCC2D73080319D42DCC2D220842
:100BF0008316A8001C2EEC220A168A152B240A1232
:100C00008A11C42DEC2265260A128A11C42DEC2209
:100C1000E822C42DEC22E422C42DEC22E022C42DD3
:100C2000DC22C42DD822C42DD422C42D0A128A1548
:100C300035210A128A11C42D83122B08F039F200D3
:100C4000F301412E72080319FB2D103A0319FB2DF5
:100C5000303A0319022E103A0319072E703A03197D
:100C60000A2E103A03190D2E303A0319102E103A9D
:100C70000319122EF03A0319142E103A0319162EE6
:100C8000CC2D73080319222ECC2D21080F3A0319FD
:100C9000622E2108033A0319622E831603173215B8
:100CA000B210542E0130632E83122608E039F20070
:100CB000F3015E2E72080319522E612E7308031978
:100CC0005A2E0313210803130800831603179401F7
:100CD0000E3095053830940640309506140883127E
:100CE0000313AD0083160317150883120313AE0018
:100CF000E2300A168A154921FF3083160317960041
:100D0000160883120313AD00E3300A168A1540213A
:100D10008316031792010E3093051F309206503050
:100D20009306120883120313AD00831603171308EA
:100D300083120313AE00E1300A168A1549210A1204
:100D40008A110F3083160317A300321BAA2E28081E
:100D5000031DAC2E0330C52EE6300A168A155E211F
:100D60000A128A11700883160317990071089A00F5
:100D70001A1DBC2E1918BE2E0F30A3002308031D08
:100D8000A52E5B23861005140B3003138312080075
:100D9000F601F401F50172087304031900341F30E1
:100DA000F6040310F60AF20DF30D031CD22EF30C19
:100DB000F20C73087102031DDF2E72087002031C0F
:100DC000E72E7208F0027308031C730AF102F40D97
:100DD000F50DF60BF61AD72EF61FF32EF409F40ACA
:100DE0000319F503F5097408F2007508F300761F7E
:100DF0000034F009F00A0319F103F1090034840109
:100E000083120313DA01F801F901FA01FB017408F6
:100E10007504760477040319102FC030DA051B2FF0
:100E2000F001F101F201F30100340310F40DF50DAE
:100E3000F60DF70DDA0AF71F152FDA0A0310F80D71
:100E4000F90DFA0DFB0D77087302031D312F76089B
:100E50007202031D312F75087102031D312F7408B2
:100E60007002031C422F78147408F0027508031CEA
:100E7000750FF1027608031C760FF2027708031C47
:100E8000770FF3020310F70CF60CF50CF40CDA03F1
:100E90005A083F39031D1E2F5A1F5B2F0310FF30C6
:100EA000F007F009031CF107F109031CF207F2092E
:100EB000031CF307F3097008F4007108F5007208C9
:100EC000F6007308F7007808F0007908F1007A0856
:100ED000F2007B08F300DA1FB52F0310FF30F00794
:100EE000F009031CF107F109031CF207F209031CC6
:100EF000F307F309B52F84017008F8007108F900B1
:100F00007208FA007308FB00F201F301F001F1012D
:100F10000310FB0CFA0CF90CF80C031C9D2F740841
:100F2000F00775080318750FF10776080318760F98
:100F3000F20777080318770FF307780879047A0423
:100F40007B040319B52F0310F40DF50DF60DF70D05
:100F5000882F0008F000840A0008F100840A0008C5
:100F6000F200840A0008F3007C2F8408031900347F
:100F70007308800084037208800084037108800075
:100F80008403700880000034003400342B340D34A6
:100F90000A340834023432340234063407340A3452
:100FA000143400348A340034003400341E340234E3
:100FB0000034C134403400340134B03430340034AF
:100FC00000340034053400342B340D340A34083432
:100FD0000234323402340634073414341434003406
:100FE00080340034003400341E3402340034C13400
:100FF000003400340334B034B034003400340034EE
:10100200F0000030711870070310F00D0310F10C9E
:10101200F108031D0328080083120317281C142853
:101022008316111616288316111211149017100820
:1010320083120313AD0083160317110883120313DF
:10104200AE00E0300A168A15492114300A168A11B8
:101052000820831603179013100883120313AD00A0
:1010620083160317110883120313AE00E0300A1629
:101072008A15492983120313A20083160317A300BA
:1010820005300A168A1108200A128A1583160317D8
:10109200321B4E282808031D502803306C28E630E6
:1010A2000A168A155E210A128A157008831603171A
:1010B200990071089A001A1D6228991F62281A1C49
:1010C200682883120313220883160317A300230838
:1010D200031D4128003003138312080083160317EF
:1010E20094010E3095053830940650309506140858
:1010F20083120313AD00831603171508831203131B
:10110200AE00E2300A168A1549210A128A150C30FD
:101112003B200038031DC628861005144D30831667
:101122000317A300321BC62828080319C62820303B
:10113200230203189328FF30960016088312031324
:10114200AD00E3300A168A15402183160317920177
:101152000E3093051F309206403093061208831218
:101162000313AD0083160317130883120313AE0093
:10117200E1300A168A1549210A128A1583160317C5
:10118200321BC6282808031DC8280330CF2823088D
:10119200031DC1280A128A115B230C300313831228
:1011A20008008316031794010E3095053830940613
:1011B20070309506140883120313AD0083160317CB
:1011C200150883120313AE00E2300A168A1549216C
:1011D2000A128A1505303B200038031D2929861082
:1011E20005144D3083160317A300321B2929280842
:1011F20003192929203023020318F628FF3096000C
:10120200160883120313AD00E3300A168A15402133
:101212008316031792010E3093051F309206603039
:101222009306120883120313AD00831603171308E3
:1012320083120313AE00E1300A168A1549210A12FD
:101242008A1583160317321B29292808031D2B2907
:10125200033032292308031D24290A128A115B2331
:101262000A300313831208008316031794010E3009
:1012720095053830940660309506140883120313DE
:10128200AD0083160317150883120313AE00E23074
:101292000A168A154921FF3083160317960016088D
:1012A20083120313AD00AE01E3300A168A154921F9
:1012B2008316031792010E3093051F309206703089
:1012C2009306120883120313AD0083160317130843
:1012D20083120313AE00E1300A168A1549210A125D
:1012E2008A1505303B20003803197929033008009C
:1012F2000A128A115B23861005140A348316031717
:10130200B50A902983120313A2019F29C0308A29AA
:10131200803083120313A2009F290430A7293508C5
:10132200C03E840083170008303A03198329013A2A
:1013320003198729033A031989298E293F30031794
:10134200A705031322080317A7060030031383120D
:10135200080083160317B50AB9290030B1290130F4
:101362000A168A1194260A128A15C5290430C6293A
:101372003508C03E840083170008303A0319AE29AD
:10138200013A0319B029B729003003138312080068
:1013920083160317B50AD129AA21E3297F21E3295C
:1013A2003508C03E840083170008463A0319CD2948
:1013B200013A0319CF29213A0319CD29013A031918
:1013C200CF29043003138312080083160317B50ACA
:1013D200442BB50A83120313A301A30AA401A40A8E
:1013E2003C2AE03083120313A60090303A2AE130FF
:0E13F20083120313A60092303A2AE2308312CF
:101400000313A60094303A2A83120313A301E33096
:10141000A6009630192A83120313A301E430A60014
:101420009730192A83120313A401A301E530A60003
:101430009830A2006B2A83120313A401E630A600A1
:1014400099303A2AE83083120313A6009B303A2AD7
:10145000E93083120313A6009D303A2AEA30831242
:101460000313A6009F303A2A83120313A401EB3022
:10147000A600A130A5006B2A831603173508C03ECD
:10148000840083170008303A0319F229013A03193E
:10149000F829033A0319FE29013A0319042A073AE5
:1014A00003190B2A013A0319122A033A03191B2ABA
:1014B0000E3A0319222A013A0319282A783A031905
:1014C0002E2A033A0319342A233A03192E2A033AFF
:1014D0000319342A422B83160317B50A3508C03E78
:1014E0008400831700083D3A031DD52A8312031395
:1014F000A408831603170319D72AB50A9C24700879
:10150000A9007108AA007208AB007308AC00003093
:101510002C02031D952A01302B02031D952A003051
:101520002A02031D952A003029020318422BA30822
:10153000031DAA2A00302C02031DA82A00302B020A
:10154000031DA82A01302A02031DA82A00302902FF
:101550000318422BA3080319C42A25088400831703
:1015600029088000840A2A0880002508840083173F
:101570000008AD00840A0008AE0026080A168A1585
:1015800049210A128A15562B22088400831729083C
:1015900080002208840083170008AD0026080A1680
:1015A0008A1540210A128A15562B8316031735080F
:1015B000C03E8400831700083F3A031D422B83126C
:1015C0000313A3080319FE2AA408031DF52A2608FD
:1015D0000A168A155E210A128A15250884008317C7
:1015E00070088000840A7108800025088400831731
:1015F0000008A700840A0008A800132BA408031DF4
:101600000D2B26080A168A1554210A128A15F00095
:101610002208840083177008800022088400831742
:101620000008A700A80103171E1E292B0313270873
:10163000BB002808BC000430BD00003003179E1911
:1016400001300313BE000A168A1596260A128A155F
:10165000562B03132708BB002808BC000530BD002B
:10166000003003179E1901300313BE000A168A15B5
:1016700005260A128A15562B0A168A1573210A1294
:101680008A15562B0430572B3508C03E840083172B
:101690000008453A0319EA29173A03193C2B373A4F
:1016A0000319EA29173A03193C2B422B0030031384
:1016B0008312080083160317B50AE92B1030831232
:1016C000031385000630860400300A168A11DC24D4
:1016D0000A128A1583160317B312082C0F308312CF
:1016E00003138500F930860501300A168A11DC24BF
:1016F0000A128A1583160317B316082C64300A16CB
:101700008A1108200A128A15082C01300A168A113B
:1017100019200A128A15082C8B1283122510932B7C
:101720008B128312251483163B14082C3216082CB6
:101730001E30A80083120313061CA42B8316031764
:101740002808031D9A2BE72BE6300A168A155E211E
:101750000A128A15700883160317990071089A00F7
:1017600083121E1ECC2B8316190883120313BB0091
:10177000831603171A0883120313BC000430BD003C
:10178000003003179E1901300313BE000A168A1594
:1017900096260A128A15082C831619088312031339
:1017A000BB00831603171A0883120313BC0005300D
:1017B000BD00003003179E1901300313BE000A1646
:1017C0008A1505260A128A15082C0F30092C0430B8
:1017D000092C3508C03E840083170008F000303023
:1017E000F002031CE72B0A3070020318E72B0B30C2
:1017F0008A00FE30700703188A0A82005E2B6E2B67
:101800007E2B852B8C2B902B962B982BE52BE52B69
:10181000003003138312080083160317B50A142C33
:101820005A23262CE621262C3508C03E8400831737
:101830000008463A0319102C143A0319122C343AB2
:101840000319102C143A0319122C043003138312B9
:10185000080083160317B50A382C0030302C0130ED
:101860000A168A1194260A128A15442C0430482C30
:101870003508C03E840083170008303A03192D2C28
:10188000013A03192F2C362C0A168A1573210030C1
:1018900003138312080083160317B50A602C831202
:1018A0000313A201752C80305A2CA0305A2CC03062
:1018B0005A2CE03083120313A200752C04307D2CC7
:1018C0003508C03E840083170008303A03194F2CB6
:1018D000013A0319532C033A0319552C013A031901
:1018E000572C073A0319592C5E2C1F300317A605F5
:1018F000031322080317A6060030031383120800FF
:1019000083160317B50A8C2C83129E11982C831210
:101910009E15982C0430992C3508C03E84008317FE
:101920000008303A0319842C013A0319872C8A2CB9
:10193000003003138312080083120313B301B401B0
:10194000B501B601AF01AF0AB001B101B201AE01FC
:10195000BD2C831603173508C03E8400831700088A
:10196000F000831203132E08373E8400831370089F
:101970008000AE0A83160317B50A831603173508CD
:10198000C03E840083173A3000020318D62C350875
:10199000C03E8400831730300002031CD62C831213
:1019A00003132E08803A7A3E031CA92C83160317D2
:1019B000B50383120313AE032E08AD00AD1B1C2D1F
:1019C0002F08F4003008F5003108F6003208F7005F
:1019D0002D08373E840083130008F000F101D03059
:1019E000F0070318F10AFF30F107700871080030A2
:1019F000F11BFF30F200F3000A128A117B277008F6
:101A0000B30771080318710FB40772080318720F37
:101A1000B50773080318730AB6070A30F400F50116
:101A2000F601F7012F30840083130A128A11A927C7
:101A30000A128A15AD03DE2C3308F0003408F100D9
:101A40003508F2003608F300080083120313A301DF
:101A500083160317B50A3508C03E840083173A3051
:101A600000020318E82D3508C03E8400831730308B
:101A70000002031CE82D3508C03E840083170008CF
:101A8000F000831203132308253E8400831370089B
:101A90008000A30A83160317B50A3508C03E8400E8
:101AA00083173A30000203186F2D3508C03E8400BA
:101AB000831730300002031C6F2D3508C03E8400B0
:101AC00083170008F000831203132308253E8400C7
:101AD000831370088000A30A83160317B50A8312C4
:101AE00003132308253E8400831380012530AC00B6
:101AF0008030AD000A168A15B4220A128A157008C1
:101B0000A2001E3022020318E82D1030A400220883
:101B1000A407831603173508C03E84008317000806
:101B20003D3A031DB32DB50A9C247008A800710826
:101B3000A9007208AA007308AB0000302B02031D35
:101B4000AB2D00302A02031DAB2D01302902031DED
:101B5000AB2D003028020318E82D240884008317D9
:101B600028088000EA2D3508C03E8400831700084D
:101B70003F3A031DE82D83121E1ED32D03132408A4
:101B8000840083170008BB00BC010230BD00003098
:101B900003179E1901300313BE000A168A159626F4
:101BA0000A128A15EA2D03132408840083170008FB
:101BB000BB00BC010330BD00003003179E1901308B
:101BC0000313BE000A168A1505260A128A15EA2D85
:101BD0000430EB2D00300313831208008316031723
:101BE000B50AFA2D83121E11062E83121E15062E1B
:101BF0000430072E3508C03E840083170008303AB1
:101C00000319F22D013A0319F52DF82D00300313B5
:101C100083120800831603173215B2101030031315
:101C20008312080083160317B50A1C2EB211282E42
:101C3000B215282E0430292E3508C03E84008317A3
:101C40000008303A0319162E013A0319182E1A2EDD
:101C5000003003138312080083160317B50A592EA8
:101C60000030512E0130512E02300A168A11E4251F
:101C700009300A168A11E42505300A168A11E4256E
:101C80000A128A150830512E03300A168A11E425EB
:101C90000A128A150630512E04300A168A11E425DC
:101CA00007300A168A11E4250A128A156E2E0430AE
:101CB0006F2E3508C03E840083170008303A0319A0
:101CC000302E013A0319322E033A0319342E013A09
:101CD0000319442E073A03194C2E572E00300313D4
:101CE0008312080083160317B50A812E0030792E5F
:101CF00001300A168A11DC240A128A158D2E04304E
:101D00008E2E3508C03E840083170008303A031930
:101D1000762E013A0319782E7F2E0030031383129A
:101D2000080083160317B50A9D2E83129E10A92E54
:101D300083129E14A92E0430AA2E3508C03E8400BA
:101D400083170008303A0319952E013A0319982E8B
:101D50009B2E003003138312080083160317B50A65
:101D60003508C03E84008317000883120313A300C4
:101D70004C3A0319BF2E23086C3A031DC52E0317D6
:101D800030080319182F8316132FA201E02E220802
:101D9000303E8400831723088000A20A10302202FC
:101DA000031CD52E0317B001182F83160317B50A8D
:101DB0003508C03E84008317000883120313A30074
:101DC0003A3023020318E82E303023020318C72EBE
:101DD000453023020318F02E413023020318C72E8A
:101DE000653023020318F82E613023020318C72E32
:101DF0002308233A0319C72E23082A3A0319C72EAA
:101E000023082C3A0319C72EA2080319182F83168A
:101E10000317B503831203132208303E840083178F
:101E2000800183160317B21083129E171030192FEA
:101E300004300313080083160317B50A3A2F8312E0
:101E40000313A201592F1030342F2030342F30309B
:101E5000342F4030342F5030342F6030342F7030D6
:101E6000342F8030342F903083120313A200592F67
:101E70000430612F3508C03E840083170008F0004D
:101E80003030F002031C382F0A3070020318382F4C
:101E90000F308A004F30700703188A0A82001F2F04
:101EA000232F252F272F292F2B2F2D2F2F2F312F6A
:101EB000332F0F300317AB05031322080317AB06AC
:101EC000003003138312080083160317B210831225
:101ED0009E1310300313080083160317B501F52F66
:101EE0006427EC2F1B27EC2FAD26EC2F9126EC2F2F
:101EF0007226EC2F2C26EC2F1226EC2F0A26EC2F24
:101F0000EE25EC2F2525EC2F8024EC2F4B24EC2FF5
:101F100029240A128A15EC2FC921EC2F0C24EC2F4E
:101F20003508C03E840083170008263A03198C2F19
:101F3000663A03198E2F013A0319702F033A0319D9
:101F4000722F063A0319742F013A0319762F0D3AAE
:101F50000319782F013A03197A2F073A03197C2FB6
:101F6000013A03197E2F1E3A0319802F023A0319F2
:101F7000822F053A0319842F0E3A0319862F023A4D
:101F80000319882F3B3A0319702F033A0319722F54
:101F9000063A0319742F013A0319762F0D3A0319E3
:101FA000782F013A03197A2F073A03197C2F013A47
:101FB00003197E2F1E3A0319802F023A0319822F2C
:101FC000053A0319842F0E3A0319862F023A031992
:101FD000882F043083120313A100A1080319F22FE4
:101FE0002108FD2F83160317B50A3508C03E84006B
:101FF00083170008031D902F00300313831208007D
:1020000083120313A0000C1E032820089900080067
:1020100083120313A500A508031908000430A600C5
:102020005330A700A70B1228A60B1028A50B0E28CB
:10203000080083120313A200A20803190800043049
:10204000A300FA300820A30B2128A20B1F280800A8
:10205000831603171A1D3028911C3028B4113C2810
:10206000B41D37283008031D3C2801303D28B41525
:1020700083121A088316B00000300313831208007D
:1020800083160317B801B90183121C088316A9002F
:102090003410B410341180309005FF309105493070
:1020A0009006100883120313AD008316031711085E
:1020B00083120313AE00E0300A168A1549210A166E
:1020C0008A11143083160317AE003608370603133F
:1020D000031D0C1603173908380603198E28341E01
:1020E000912803138C1203173908403E840083178C
:1020F00000089600B90A160883120313AD00E330F6
:102100000A168A1540210A168A110F308316031702
:10211000B90503138C160317341291288312031385
:10212000861383120313061C9A28831603172E089E
:10213000031DD1288B13E6300A168A155E210A1674
:102140008A11700883160317990071089A00191FE5
:10215000BB28E5300A168A1554210A168A11F000A8
:10216000831603173608503E8400831770088000DA
:10217000B60A1F30B6051A1E9A19341628200038E0
:102180000319CD280A168A1573210A168A1105101B
:102190008614831603173211B214143083160317F2
:1021A000AE008B17B21C652880309005FF3091057A
:1021B000100883120313AD0083160317110883124E
:1021C0000313AE00E0300A168A154929831603135B
:1021D0008112811112300317BE00132983160313D5
:1021E00001118110011024301029831603130115E9
:1021F0008110011401301029831603130111811479
:1022000001100930102983160313011181140114E0
:1022100005301029831603130115811001100330B6
:102220000317BE00352983122B08F039F200F301A1
:102230002C2972080319EE28203A0319F528603A70
:102240000319FC28103A03190329203A03190A2913
:10225000E03A031903292F29730803191929831652
:10226000031301118110011403173E08973E8312D6
:10227000031381000B118B1608000A168A157321AF
:102280000A128A150D200A168A110317A81C4B2959
:10229000831611154D29831611111008831203138B
:1022A000AD0083160317110883120313AE00E0304C
:1022B0000A168A154921FF3083160317960016085F
:1022C00083120313AD00E3300A168A1540210A1663
:1022D0008A110E2A0030251C75298316920640307B
:1022E00093060030940650303E2A83169406403000
:1022F0009506003092065030E9290030251C8829C7
:1023000083169206503093060030940640303E2AE1
:102310008316940650309506003092064030E92925
:10232000251C9429A51898292518A129A518A129A3
:10233000003083169206B030930600309406A03029
:102340003E2A003083169206A03093060030940691
:10235000B0303E2A251CAE29A518B2292518BB2964
:10236000A518BB29003083169206903093060030E2
:10237000940680303E2A0030831692068030930601
:102380000030940690303E2A0030251CCF29831659
:102390009206203093060030940630303E2A831691
:1023A000940620309506003092063030E92900303E
:1023B000251CE229831692063030930600309406DD
:1023C00020303E2A8316940630309506003092065F
:1023D000203093063F2A251CEF29A518F32925183C
:1023E000FC29A518FC29003083169206703093064C
:1023F0000030940660303E2A00308316920660302A
:1024000093060030940670303E2A00308316920600
:10241000C030930600309406D0303E2A03172B08B4
:10242000F039F200F3012B2A7208203A03196A29C5
:10243000103A03197D29703A03199029103A0319AB
:10244000AA29203A0319C429F03A0319D729103AC6
:102450000319EB292E2A73080319142A251C322A82
:10246000A518362A2518052AA518052A003083162E
:102470009206D030930600309406C0309506831241
:102480002908F000F1010930F2000310F00DF10D00
:10249000F20B452A0030F0050E30F1057008831666
:1024A00092067108930683122A08F000F1010930A0
:1024B000F2000310F00DF10DF20B592A0030F00577
:1024C0000E30F10570088316940671089506852A6A
:1024D000A51C792A2708F000F1010310F00DF10D79
:1024E0008030F0050130F1057008831692067108FE
:1024F000930603108312250C60398316920683120B
:102500002508C039831694069B2A83122B08F039BC
:10251000F200F301982A72080319682A103A031985
:10252000682A503A0319682A203A0319682A9B2A14
:10253000730803198B2A1F308316920638309406CD
:10254000120883120313AD008316031713088312B6
:102550000313AE00E1300A168A15492183160317CA
:10256000140883120313AD00831603171508831292
:102570000313AE00E2300A168A1549210A168A11A1
:10258000392B251CCA2A02300A168A1119200A166C
:102590008A11E42AE6300A168A155E210A168A1183
:1025A000700883160317990071089A00321B4F2B8D
:1025B00032300A168A1108200A168A118316031768
:1025C0001A1DCA2A991FCA2A831203172B08F03929
:1025D000031D222BFF30831692050F309305FF3029
:1025E00094050F3095058312251CF82AA518FC2A9E
:1025F0002518052BA518052B003083169206F03000
:10260000930600309406E0300D2B003083169206BE
:10261000E030930600309406F030950612088312DD
:102620000313AD0083160317130883120313AE00C0
:10263000E1300A168A1549210A168A1183160317F2
:102640001514282B281D262B8316202B83161510D6
:10265000140883120313AD008316031715088312A1
:102660000313AE00E2300A168A1549210A168A11B0
:102670004F2B03172B08F039F200F3014C2B720893
:102680000319C12A103A0319C12A503A0319C12A61
:10269000203A0319C12A4F2B730803193F2B031348
:1026A0008312080028308316031385008312080064
:1026B000522383160317321D8A2BE0309205FF3018
:1026C00093051F309206120883120313AD00831680
:1026D0000317130883120313AE00E1300A168A159C
:1026E0004921C730831603179405FF30950538300C
:1026F0009406140883120313AD00831603171508FC
:1027000083120313AE00E2300A168A1549210A1615
:102710008A118B2B3D21831603179001FF30910501
:102720008312251C952B4830962B4130831690063A
:10273000100883120313AD008316031711088312C8
:102740000313AE00E0300A168A1549210A168A11D1
:10275000E6200317251CE42B8316BD01FF308312EE
:102760000313AD00E3300A168A1540210A168A11B8
:10277000831203130618DF2BE6300A168A155E2132
:102780000A168A11700883160317990071089A00B7
:1027900083160317BB18D22B0A168A15C6210A16F0
:1027A0008A11C82B160883120313AD00E3300A16F2
:1027B0008A1540210A168A1183160317BB10831647
:1027C0000317321B272CB82B03130514E6300A1607
:1027D0008A155E21700883160317990071089A0004
:1027E000E5300A168A1554210A168A118316031732
:1027F00098000830BC003B1183120313061C062C02
:10280000232C0A168A15D5210A168A118316031756
:102810003B1D012CE6300A168A155E2170088316CE
:102820000317990071089A00E5300A168A15542199
:102830008316031798000830BC003B110A168A154E
:10284000D5210A168A1183160317321FFC2B3B1061
:10285000321303138312080083120313A10183169A
:10286000031792010E309305003092061030930644
:10287000D22C2108303E8400831700082C3A031D17
:10288000492C031718080A168A1119200A168A11EA
:10289000D12C10308316031792065D2C0D30592C65
:1028A0000E30592C0F30592C0B30592C0C30592C20
:1028B0000A308316031792069A2C831203132108F9
:1028C000303E840083170008233A0319562C093A36
:1028D0000319542C1A3A0319582C713A03194E2C27
:1028E000033A0319502C013A0319522C073A0319E1
:1028F000982C253A03194E2C033A0319502C013A0F
:102900000319522C073A0319982C2108303E8400F1
:1029100083170008F000F101D030F0070318F10A26
:10292000FF30F107700883160317920671089306AB
:1029300083160317120883120313AD0083160317BF
:10294000130883120313AE00E1300A168A154921D9
:102950000A30F10003171B080A128A1501200A1613
:102960008A110820831603179201FF30930512087D
:1029700083120313AD008316031713088312031386
:10298000AE00E1300A168A1549210A30F10003171A
:102990001B080A128A1501200A168A1108200A1635
:1029A0008A11A10A831203132108303E8400831781
:1029B000000803190800392C83120313A200A2088F
:1029C00083160317031DE62C9110E72C91141008B1
:1029D00083120313AD008316031711088312031328
:1029E000AE00E0300A168A154929831603172E080F
:1029F000031D572D1430AE00B21B172DBA01E6305F
:102A00000A168A155E210A168A11700883160317A2
:102A1000990071089A001A1F572D8312910183168D
:102A2000BA0AAF01B2178312031306110800473028
:102A30002F020318572DE6300A168A155E210A1652
:102A40008A11700883160317990071089A001A1FDB
:102A5000332D831203130611831603173A0A031941
:102A6000572DBA0A572D8312031306150F308316FC
:102A700003173A02031C542D8312910A02300A16DE
:102A80008A15F7260A168A11031711081006031D66
:102A90004F2D8316B213B21083129E13572D503050
:102AA0008316AF00BA01572D2F080319B213031371
:102AB00083120800E6300A168A155E210A168A116A
:102AC000700883160317990071089A009A1E5A2DF0
:102AD000183083120313AD00C030AE00E9300A167F
:102AE0008A154921E6300A168A155E210A168A11CE
:102AF000700883160317990071089A009A1E722DA8
:102B0000E5300A168A155E210A168A11710A5430B8
:102B10000319700603198E2D04300800E6300A16DA
:102B20008A155E210A168A11700883160317990008
:102B300071089A009A1E8E2DEB300A168A155E21B6
:102B40000A168A117108673AA13003197006031931
:102B5000AB2D04300800E6300A168A155E210A16ED
:102B60008A11700883160317990071089A009A1E3B
:102B7000AB2DE5300A168A155E210A168A117108F6
:102B8000FE3A3530031970060319C82D04300800C9
:102B9000E6300A168A155E210A168A117008831615
:102BA0000317990071089A009A1EC82DEB300A1677
:102BB0008A155E210A168A1171082C3A8030031991
:102BC000700603190034043483120313A200A30116
:102BD00003171E19742E1F2E2530BC000230172E2D
:102BE000C530BC000030172E5A30BC000130172E03
:102BF0002E30BC000130172E7A30BC000130172E69
:102C0000F030BC000030172E1830BC000130172EF9
:102C1000DE30BC000030172EC830BC000130172E4B
:102C20000530BC000130172E8630BC000130BD00DD
:102C300024300A168A15AC200A168A114C2E03136A
:102C40002208F0000B3070020318080016308A00CA
:102C50002D30700703188A0A8200EC2DF02DF42D18
:102C6000F82DFC2D002E042E082E0C2E102E142EC6
:102C70002308243E840083130008F0008316031702
:102C80003608503E8400831770088000B60A1F3053
:102C9000B60583120313A30A2308243E840083137A
:102CA0008008031D382E831603173608503E840013
:102CB00083178312130880008316B60A1F30B605E7
:102CC00083129E1D6F2E83163608503E8400831794
:102CD0008312140880008316B60A1F30B6058316C7
:102CE00003130C160C1A722E03138312080083169A
:102CF0000317A901AE01AF01A301A401A501A6011B
:102D0000A701A8010A30AB00AC00AD003230AA0028
:102D100003138112811101118110011416308312E5
:102D200081000B118B16080083120313A2000230DE
:102D30002202031808001030A300A4011E30F10085
:102D400022080A128A1501200A168A112407A03EB9
:102D5000840083130008F0002308840083177008A0
:102D60008000A30AA40A1E302402031808009E2E25
:102D700083120313A1012108C03E84008317800140
:102D8000A10A30302102031CBB2EA1012108503EB4
:102D9000840083178001A10A20302102031CC62E63
:102DA0000317B0018316B201B301BB01B401B50131
:102DB000B601B701B801B90103138312080030301E
:102DC0008316031385007130860093308700063028
:102DD0009F0083128501AC3086004C3087000800CC
:102DE000831603138101830183128C018B018316E7
:102DF0008C0183120800F026DF26B82600309426C6
:102E00000A168A1576200A168A1573210A168A115F
:102E10007726A1014B30A2000030A301A401A50137
:102E20000A128A1135220A168A110B178B1783167C
:102E30008C168312061A1A2F86110030E4250A1206
:102E40008A150D200A168A115A25043A031D2A2FC5
:102E50000A30E4250A168A1573210A168A11831688
:102E600003173214B214831203138613831203134D
:102E7000061A3C2F05153D2F0511831603173B1C21
:102E80004E2F0A168A1158230A168A1177260A1617
:102E90008A1553200A168A1183160317321E5B2FD8
:102EA0000A168A15B8270A168A1183160317321FC5
:102EB000502F32123213B21C642F831210080319E0
:102EC000622FF52483160317331E6C2F03130C1A7D
:102ED000672F0C1603173312B31D7D2F0A128A15A4
:102EE0006C270A168A15F7260A168A118316031705
:102EF000B311B50183120313861383160317321916
:102F0000B52FB218B52F0A168A15E3210A168A11B1
:102F10000130DC240A168A1103179E1F962F16080B
:102F20000A168A1119200A168A112C240A128A11EB
:102F3000A925A0000A168A15F7260A168A11200864
:102F4000033A0319A72F20080F3A031DB32F0A16BF
:102F50008A1573210A168A11051086148316031721
:102F60003211B214321383160317321DD12FB21847
:102F7000D12F0A168A1140200A168A1183160C1ABC
:102F8000BF2F83128613831603173219C92F0330FC
:102F9000CA2F00300A168A15F7260A168A118316D8
:102FA0000317321DFB2F2E08031DFB2FE6300A16D8
:102FB0008A155E21700883160317990071089A001C
:102FC0000A168A1128200A168A1100380319F72FC9
:102FD0000A168A15732105108614831603173211F9
:102FE000B21403300A168A15F7260A168A1114300D
:102FF00083160317AE003218362F0A128A11992849
:1030A600303083160313850083120800831203133E
:1030B6008C1E5B281A08080083120313981C003420
:1030C600181218160134831203138C1E6828003058
:1030D600181901300800831203138C1E7028003063
:1030E6001818013008008312031394011412831672
:1030F6001417831294168C110800F400F40AF403D2
:10310600031900340310F00DF10DF20DF30D8228B2
:1031160083120313B1003A30310203189528303078
:103126003102080003100800F401F5010310F30C46
:10313600F20C031CA4287008F40771080318710A1E
:10314600F5070310F00DF10D72087304031D99289D
:10315600003483120313BE00BF003D08CC003C08B8
:10316600BC0A0319BD0A0A128A11B3200A168A1567
:10317600F000BF0A3F0384008313700880008008B4
:10318600031DB0283E080800831203130C1E080016
:10319600061B080083160317370836060319E128AD
:1031A6003708503E840083170008831203139900E2
:1031B60083160317B70A1F30B705E32803130C124B
:1031C6000313831208008B1283160317AA032E0813
:1031D600031DAE032A08031DF5283230AA0029086C
:1031E600031DA903AB0B2F290A30AB00AC03230840
:1031F600031DA3032408031DA4032C08031D2F2964
:103206000A30AC00AD033008031DB0032F08031DC0
:10321600AF032508031DA503260803191429A603D1
:103226002429B31E1C2983120313851585148316BE
:103236000317B31A242983120313851185108316E5
:1032460003172D08031D2F290A30AD002708031D7B
:10325600A7032808031DA803163083120313810051
:103266000B118B16080083120313B2003208930069
:103276008C1D3B298C111308080083120313AE0022
:10328600071136212D08362107150800831203136E
:10329600AF00071136212E0836212D0836210715D5
:1032A600080083120313AD000711362100303621C2
:1032B600AE000715080083120313AD00071136216F
:1032C60000303621AF0000303621AE0007152F083A
:1032D600B1002E08B0003108F1003008F0000800F7
:1032E60083120313071101303621071583160317BE
:1032F6009001910192019301940195019601970124
:103306009B019C019D019E019F01A0010313831255
:103316000800031083160317980C83120313031C6B
:1033260085100318851483160317BC033C0803197C
:103336003B150313831208008312031305110310B0
:1033460083160317BD0CBD1383120313851DAF2906
:10335600803083160317BD0683160317BC033C088B
:10336600031DBA293D0896000830BC00BB140313A0
:1033760083120800831603173E08973E8312031331
:1033860081000B110800BD210519CB290515D2298D
:10339600831603173C0BD129BB18D2299F2103138F
:1033A60083120800BD21051CDA290510E0298316C1
:1033B60003173B19E0298C21051403138312080017
:1033C6000A168A1573210A128A150D200A168A15FD
:1033D60003172908F000F1010930F2000310F00D7F
:1033E600F10DF20BF1290030F0050E30F1057008F1
:0A33F6008316920671089306120870
:1034000083120313AD0083160317130883120313EB
:10341000AE00E1300A168A1549210A168A150317EB
:103420002A08F000F1010930F2000310F00DF10D4F
:10343000F20B152A0030F0050E30F10570088316E6
:10344000940671089506140883120313AD008316C1
:103450000317150883120313AE00E2300A168A150B
:1034600049210A168A150317A81C392A8316111533
:103470003B2A83161111100883120313AD00831623
:103480000317110883120313AE00E0300A168A15E1
:1034900049290A168A1566200A168A150038031962
:1034A000572A0A168A1559200A168A15B12A0A16A9
:1034B0008A155920C5000A168A155F200A168A1532
:1034C0000038031DB12A831603173808403E8400D4
:1034D0008317831203134508800083160317B80A65
:1034E0000F30B8053808F000F1013908F002031C6C
:1034F000F1030F30F005F1017108803AF2008030DD
:103500007202083003197002031C8B2A8312031302
:1035100086178316031729080319341483121C080D
:103520008316A90083120313450803171206831696
:1035300003199E2A3410B4103411B12A341CB12A54
:10354000B418A42AB414B12A3419A82A3415B12AFB
:10355000B214B801B9013410B4103411831203133A
:103560008613031383120800B82AAC0A0319AD0AA4
:10357000831203132D08CC002C080A128A11B320E1
:103580000A168A15203A0319B52A2D08CC002C08F2
:103590000A128A11B3200A168A15093A0319B52AA4
:1035A000AF01B001AE012D08CC002C080A128A111F
:1035B000B3200A168A152D3A031DE02AAE0AE82A1E
:1035C0002D08CC002C080A128A11B3202B3A0319BB
:1035D000AC0A0319AD0A2D08CC002C080A128A1176
:1035E000B3200A168A158B200A168A15031C1B2B7A
:1035F0000A30F200F3013008F1002F08F0000A163B
:103600008A1597202D08CC002C080A128A11B320A5
:103610000A168A15F000F1017408F0070318F10A80
:103620007508F107D0307007AF00FF300318003085
:103630007107B000E82AAE080319282B3008F10002
:103640002F08F000F009F109F00A0319F10A080047
:103650003008F1002F08F00008000A168A156620CD
:103660000A168A15003803193B2B0A168A155920A9
:103670000A168A15282C0A168A155920C5000A161A
:103680008A155F200A168A150038031D282C831618
:103690000317B319282C3B18552B321A552BB21A85
:1036A000552BB218572B3219572B3217282C3A307A
:1036B0008312031345020318612B303045020318AF
:1036C000A12B5B3045020318692B413045020318DA
:1036D000A12B7B3045020318712B61304502031882
:1036E000A12B4508031713060319A12B0313450843
:1036F000031715060319A12B03134508263A0319CE
:10370000A12B4508403A0319A12B45083D3A03195E
:10371000A12B45083F3A0319A12B45082C3A031960
:10372000A12B4508253A0319A12B45082A3A03196C
:10373000A12B4508233A0319A12B45082F3A031D55
:10374000002C83160317B31CD72B831203134508D1
:1037500003171306031DAE2B8316BE2B0313450858
:10376000031715068316031DBA2B35080319FF2B03
:10377000B503FF2B35082F3A031DCB2B3508C03E70
:103780008400831780013315B3103310B3158312EF
:1037900003138617002C3508C03E8400831783125C
:1037A00003134508800083160317B50AFF2B331C4B
:1037B000F22B8312031345082F3A031DE62B8316C1
:1037C00003173310B3158312031386174508543AB1
:1037D0000319EE2B4508743A031D002C83160317BA
:1037E000B314FF2B831203134508413A0319FC2B32
:1037F0004508613A031D002C831603173314831206
:1038000003179E1C282C83163608503E840083170D
:10381000831203134508800083160317B60A1F306E
:10382000B60583120313450803171306031D262C40
:103830009E1D262C83163608503E84008317831263
:10384000140880008316B60A1F30B6058316331697
:1038500003138312080083120313A201A301A4011E
:103860008316031794010E309505F8309406C03086
:103870009506140883120313AD0083160317150869
:1038800083120313AE00E2300A168A154921FF3075
:10389000831603179600160883120313AD00E33056
:1038A0000A168A1540218316031792010E309305DC
:1038B00083122708F000F1010310F00DF10D8030A4
:1038C000F0050130F1057008831692067108930621
:1038D0001F309206D0309306120883120313AD00F6
:1038E00083160317130883120313AE00E1300A1680
:1038F0008A154921183083160317A30005300A16CC
:103900008A1108200A168A1583160317321BEE2D1A
:1039100028080319EE2DE6300A168A155E210A16CC
:103920008A15700883160317990071089A001A1DEA
:103930009D2C991F9D2C1A189F2C1830A3008312C0
:103940002B08F0398316031DB32CB219A92C18309B
:10395000A3001A1DB32C9A1CB32C83120313A401C9
:10396000A40A831603172308831203130319BB2C1D
:10397000A40803197E2CA4080319B52D05300A16D6
:103980008A1108200A168A1583160317321BEE2D9A
:1039900028080319EE2DE6300A168A155E210A164C
:1039A0008A15700883160317990071089A009A18EF
:1039B000BE2CF8309205FF309305120883120313D2
:1039C000AD0083160317130883120313AE00E13012
:1039D0000A168A1549210A168A153C3083160317E0
:1039E000A300321BEE2D28080319EE2D32302302DE
:1039F0000318F12C98309205FF309305673092063A
:103A0000120883120313AD008316031713088312E1
:103A10000313AE00E1300A168A1549210A168A15E9
:103A200083160317321BEE2D28080319EE2D1E30C6
:103A300023020318122D1514140883120313AD006A
:103A400083160317150883120313AE00E2300A161B
:103A50008A1549210A168A1583160317321BEE2D83
:103A600028080319EE2D0F30230203182E2DFF30E6
:103A700094050F30950500309406E0309506140843
:103A800083120313AD008316031715088312031363
:103A9000AE00E2300A168A15492105300A168A114D
:103AA00008200A168A1583160317321BEE2D2808E4
:103AB0000319EE2D83120313A308031D822D831611
:103AC00003172308031D822DFF3092050F30930545
:103AD00000309206F0309306120883120313AD00F3
:103AE00083160317130883120313AE00E1300A167E
:103AF0008A154921143083160317A3008312031378
:103B0000A301A30AE6300A168A155E210A168A1551
:103B1000700883160317990071089A001A1D9F2DCB
:103B2000991F9F2D1A1C9F2D83120313A208031D9A
:103B30009D2D86100514A201A20A831603171A1DD3
:103B40004D2D991F4D2D1A1C4D2D83120313A308C3
:103B500003194D2D83160317321BEE2D2808031968
:103B6000EE2D23080319F72DAC2D9F308316031774
:103B70009205FF30930560309206120883120313FA
:103B8000AD0083160317130883120313AE00E13050
:103B90000A168A1549210A168A150317281DD32DDE
:103BA00083161514D52D83161510140883120313CC
:103BB000AD0083160317150883120313AE00E2301D
:103BC0000A168A1549210A168A154D3083160317DD
:103BD000A300321BEE2D2808031DF02D0330022E0A
:103BE0002308031DE92D83120313861005140A12FE
:103BF0008A115B230A168A15A408031D012E0830BA
:103C0000022E073003138312080083120313BD082A
:103C10000319712E06303D020318712E3B08C100B6
:103C20003C08C200C301C30AC4010A30F200F30118
:103C30004308F0004408F1000A168A1597200A1676
:103C40008A157408C3007508C400BD0302303D0224
:103C50000318152E4408F3004308F2004208F1004F
:103C60004108F0000A128A11C8267408BF007508BE
:103C7000C000831603173608503E84008317831252
:103C800003133F08303E800083160317B60A1F3027
:103C9000B605831203134408F3004308F2004108F9
:103CA000F0004208F1000A128A11C8267008C1000B
:103CB0007108C2000A30F200F3014308F000440822
:103CC000F1000A128A11C8260A168A157408C30060
:103CD0007508C40000304402013003194302031880
:103CE0002A2E831603173608503E8400831783124A
:103CF000130880008316B60A1F30B605831203131B
:103D0000BE0883160319912E03173608503E84000F
:103D100083178312140880008316B60A1F30B60575
:103D200003130C160C1A922E83120800831203132D
:103D30003D08F0000310F00D0310700DC000FC30C2
:103D4000C0074008F2003C08F1003B08F000F20A0E
:103D5000AC2E0310F10CF00CF20BA92E70080F39E9
:103D6000BF000A303F028316031736080318C02E1F
:103D7000503E84008317831203133F08303EC72E42
:103D8000503E84008317831203133F08373E8000A0
:103D900083160317B60A1F30B60583120313C00833
:103DA000031D9F2E831603173608503E8400831789
:103DB0008312130880008316B60A1F30B6058312DB
:103DC0000313BE0883160319F22E03173608503E5C
:103DD000840083178312140880008316B60A1F30EC
:103DE000B60503130C160C1AF32E83120800831267
:103DF0000313A100A20103171E19B52F9E195B2FF3
:103E00001E1E0B2F03132108BB00BC010230BD0096
:103E1000BE019626B52F03132108BB00BC0102305A
:103E2000BD00BE010526B52F6130BC000130532F07
:103E30004130BC000130532F6830BC000130532F9B
:103E40004F30BC000130532F4930BC000130532F9C
:103E50006D30BC000130532F3C30BC000130532F7B
:103E6000DE30BC000130532F1830BC000230532F1D
:103E7000BC30BC000130532FEB30BC000130532F5D
:103E80009B30BC000130532FF730BC000130532F62
:103E9000AB30BC000130532F0730BC000230532F31
:103EA0006430BC000130BD0023300A168A15AC20F6
:103EB0000A168A158D2F03132108F00010307002A6
:103EC000031808001F308A006930700703188A0A37
:103ED0008200142F182F1C2F202F242F282F2C2F37
:103EE000302F342F382F3C2F402F442F482F4C2F6A
:103EF000502F2208233E840083130008F00083160D
:103F000003173608503E8400831770088000B60AF5
:103F10001F30B60583120313A20A2208233E840031
:103F200083138008031D792F831603173608503E2C
:103F3000840083178312130880008316B60A1F308B
:103F4000B60583129E1DB02F83163608503E84009E
:103F500083178312140880008316B60A1F30B60533
:103F6000831603130C160C1AB32F031383120800C5
:103F7000E6300A168A155E210A168A15700883161D
:103F80000317990071089A0083121E1EDC2F8316F6
:103F9000190883120313BB00831603171A08831230
:103FA0000313BC000430BD00003003179E1901301C
:103FB0000313BE009626F02F8316190883120313ED
:103FC000BB00831603171A0883120313BC000530C5
:103FD000BD00003003179E1901300313BE000526F3
:103FE000031723088316A300023023020318FA2FB5
:103FF0000230A3002308031DFA2F031383120800C5
:00000001FF
